:100000000C9446000C9463000C9463000C94630001
:100010000C9463000C9463000C9463000C946300D4
:100020000C9463000C9463000C9463000C946300C4
:100030000C9463000C9463000C9463000C946300B4
:100040000C9463000C9463000C9463000C946300A4
:100050000C9463000C9463000C9463000C94630094
:100060000C9463000C9463000C9463000C94630084
:100070000C9463000C9463000C9463000C94630074
:100080000C9463000C9463000C94630011241FBE55
:10009000CFEFD0E1DEBFCDBF11E0A0E0B1E0E4E9F9
:1000A000F2E000E00BBF02C007900D92A030B10754
:1000B000D9F711E0A0E0B1E001C01D92A030B10776
:1000C000E1F70C9412010C940000CF93DF93CDB7AD
:1000D000DEB710923B0080E480933A001092380023
:1000E000109237001092350087EF8093340080EC37
:1000F0008093320088E0809331001092230080E3E7
:1001000080932200109262001092610010926500AC
:1001100010926400DF91CF910895CF93DF93CDB714
:10012000DEB726970FB6F894DEBF0FBECDBF69834A
:100130007A838B839C8389819A81AB81BC819C016A
:10014000AD01689413F8220F331F441F551F1694F6
:10015000D1F780E094E2A4EFB0E0BC01CD010E94B1
:100160002801DA01C90101979E838D838D819E81CB
:10017000892F9927809398008D8180939900809191
:100180009A00886180939A0080919D008668809390
:100190009D0026960FB6F894DEBF0FBECDBFDF914F
:1001A000CF910895CF93DF93CDB7DEB722970FB6E7
:1001B000F894DEBF0FBECDBF80919B00882334F43E
:1001C00080919C0099279A83898302C01A821982A0
:1001D00089819A8122960FB6F894DEBF0FBECDBFFB
:1001E000DF91CF910895CF93DF93CDB7DEB72197FD
:1001F0000FB6F894DEBF0FBECDBF898380919B0000
:10020000992780729070009709F4F8CF89818093C4
:100210009C0021960FB6F894DEBF0FBECDBFDF91D4
:10022000CF910895CEEFD0E1DEBFCDBF0E94650033
:1002300060E875E280E090E00E948D000E94D200AC
:10024000898389818823D1F389810E94F300F6CFC5
:10025000A1E21A2EAA1BBB1BFD010DC0AA1FBB1FCA
:10026000EE1FFF1FA217B307E407F50720F0A21B3C
:10027000B30BE40BF50B661F771F881F991F1A94A9
:1002800069F760957095809590959B01AC01BD01D3
:04029000CF010895FD
:00000001FF
